:020000040000FA
:060000000219FD0200B32D
:03002B0002008D43
:03005B0002028717
:030073000200A0E8
:100080000406080C10182030406080A0C0C0D0C00A
:10009000E0C2CF0541E52360021523D0E0D0D03285
:1000A000C2AF53E67F7592FA7593FFC22053917FDA
:1000B000D2AF32C0D0C0E0C0F0D2D35388EFA88A0C
:1000C000A98C758A00758C0043881030331FE8C4F2
:1000D000540FFAE9C454F04AFAC3132AFAC3E833B6
:1000E000F8E933F9E82AFAE93403FB213630320F14
:1000F000C3E833E933FAE82AFAE93400FB21363061
:100100003115E875F056A4AAF0E975F056A42AFA5C
:10011000C5F03400FB2136E875F02BA4AAF0E97590
:10012000F02BA42AFAC5F03400C313FBEA13FAC378
:10013000EB13FBEA13FAC3EB94095006C3EB9403E9
:10014000501A0522E52270021522C3E522940A50B6
:1001500002417D7552007A007B00414EE52260022B
:1001600015223035067C007D042176AC31AD32306D
:100170003A04AC33AD34C3EA9CFAEB9DFB9208AE73
:100180005EAF5F303A425007203409D234219430B8
:100190003402C234303404AE60AF61203902B2346C
:1001A000C3EA33FAEB33FBA208500AEAF42401FA5B
:1001B000EBF43400FBC3EA9428FAEB9400FB5014F0
:1001C00078007A007B0021D4A208500878007A00D9
:1001D0007B00412AE52554036019202A16E55BF9C6
:1001E000EB7007C3E99A4002E9FAE53CC42AFAEB4E
:1001F0003400FBEA8EF0A4F9AAF0EB8EF0A42AFA00
:10020000C5F03400FBC3EB13FDEA13F80FEF1460E5
:1002100004C3E833F8C3E933EA33FAEB33FBDFED29
:10022000EB30E20678FF7AFF7B038852D230C3E8D6
:1002300094404002D221C3E559FC955A4003AC5A80
:10024000C3EC95525008EC75F004A4FAABF0EAF454
:10025000F8EBF45403F9C3E8940FFAE99400FB5067
:10026000047A007B00885489558A568B5775230A77
:10027000D0F0D0E0D0D053F7DF43F7403275230AF7
:10028000D0F0D0E0D0D032C0D0C0E0D2D3A8F9E5D1
:100290005830E007E5FA30E10741D5E5FA30E135BD
:1002A000C3E55513F8E55413F5FB88FCC3E5571374
:1002B000F8E55613F5E988EA85555853F7BFC3E5C5
:1002C000529401400575530041D5E5532401F5537F
:1002D00050037553FF53F7DFD0E0D0D0327901805F
:1002E0001479038010790A800C791E800879648063
:1002F0000479C880007817E4D5E0FDD8FAD9F62251
:100300007A147B7880127A107B8C800C7A0D7BB407
:1003100080067A0B7BC880007902E4C292D5E0FDAA
:10032000D293D5E0FDC293D5E0FDD292D5E0FDE9B0
:1003300020E002D29530E002D291E562D5E0FDE9FD
:1003400020E002C29530E002C2917496D5E0FDD95A
:10035000C9EAF8D5E0FDD8FBDBBEC2922278FFC225
:100360002120283D202912D221C3E548940A4009C2
:10037000C3E55294405002C22179A1E76023E548C9
:10038000601F74FF8548F084853FF030290375F0C5
:1003900005A4F8C5F0600278FFC3E8955B5002A899
:1003A0005B885A22C3E54794E4E5489400E55A5037
:1003B000031461B5046002F55A2275E89022055CC9
:1003C000C3E55C94084055E5E820ECF2A8BDA9BE61
:1003D000755C00E9FA79A0E76041EA7006E55D60C6
:1003E00018800CC3E8955D600EE55D5005600A1449
:1003F00080070460FA8002E55DF55DC394F6401B5A
:100400007559C0C394064013755980C39406400BB8
:10041000755940C39406400375590022E5592410CC
:10042000500274FFF55922743279A687F0A4C5F002
:10043000A2F733F8C3E895594002A859885B2275A2
:1004400047007548F022C2AF75C800A8CCA9CDAA54
:100450004130CF010A75C804D2AFAB42AC438842E9
:100460008943C3E89BF8E99C202808F9302C02A1B5
:100470005281AFAD448A44F9EA9DFA600478FF796D
:10048000FFAE45AF468B458C46A842A943C3E89EC4
:10049000F8E99FF9C3E54813FBE54713FAE82AF5A5
:1004A00047E93BF54850067547FF7548FF81F9AAB3
:1004B00047AB48AC47AD487E047F02C3EB94044091
:1004C0000A1E1FC3EB940840021E1FC3ED13FDEC70
:1004D00013FCDEF7C3EA9CFAEB9DFBEF6009C3E96E
:1004E00013F9E813F8DFF7EA28FAEB39FB8A478BB0
:1004F0004850067BFF8B478B48C3EB94025002D2D7
:100500002C3028047F03A1247892E6FFC3E53D94B4
:100510008240110FC3E53D94A040010FC3EF940644
:1005200040027F057E02E548C4540FF9E548C454F3
:10053000F0F8E547C4540F28F8C3E89EFAE99400A0
:10054000FB4009C3EA9401EB940050047A01E4FBF8
:10055000A19EAA47AB48EBC4FEEAC4540F4EFCC3AD
:10056000EA9CFAEB9400FBC3E813C313F8EA28FAF9
:10057000EB3400FB8A478B48C3EB94024002C22C49
:100580007802EBC4FE7B00EAC4540F4EFAC3EA982B
:10059000FA4005C3940150027A017892E6FF3020B8
:1005A0000280FB854E92854F93D22043E680C3E4C0
:1005B0009AF8E49BF9302C02C129E8FAE9FBD3E967
:1005C00013FDE813FC884E894FC3EF94036037EFA7
:1005D00020E00CE82CF8E93DF9ECFAEDFB8013E89B
:1005E00028F8E939F9C3E82401F8E93400F97AFF79
:1005F0007BFFC3EF9403400E8A508B51884A894B8E
:100600008C4C8D4DC15D885089518A4A8B4B8C4CE6
:100610008D4D3028127550F07551FF754CF0754DA9
:10062000FF754EF0754FFFC15DE8FAD3E813FC8803
:100630004EC3EF94036020EF20E007E82CF8ECFABB
:10064000C149E8282401F87AFFC3EF940340088ADF
:1006500050884A8C4CC15D88508A4A8C4C302002AC
:10066000C15D753A02D22043E680E525540360342B
:10067000A847A948C3E913F9E813F8C3E913F9E84F
:1006800013F8302804E92440F9C2AF53E67F75918E
:1006900000C3E498F594E499F595759104D220434C
:1006A000E680D2AF22D222754900752000302B039C
:1006B000752040800ED222754900752040302B03F2
:1006C00075200078017901202C20E5255403600273
:1006D000C2227914E548C313700104F8C39414408E
:1006E000027814302804781B791B202010E549601B
:1006F0000C302803D53A04D224E165D1650549E5DB
:100700009B5440B52002E14F30280908C3E89940C6
:100710000118C1EA20220A08C3E8994002C1C3C1F6
:10072000EAC222C2AF53E67F759100302C12759455
:10073000007595FE759104D22043E680D2AFC1C307
:10074000AE47AF48C3E49EF594E49FF595E134C30A
:10075000E53994015002C1C3302202C1C3D802E17D
:1007600063C1EAC224C2AF53E67F759100855094FD
:10077000855195759104854A92854B93D22043E625
:1007800080D2AFE525540360072029020539801087
:1007900030240D202B0A20220715811581020E70AE
:1007A0002278003021053022027801E53D75F007FE
:1007B000A4F9E5F028F5F0E9A2F013A2F113A2F2F2
:1007C00013F53DC394785003753D78C3E53D953EE0
:1007D000400BD223C295C293C29175D53F302002FF
:1007E00080FB854C92854D93D22043E680222038B1
:1007F00010C2AFC292D29475D53CD2AF759F200182
:10080000C2C2AFC292D29075D50FD2AF759F2001F0
:10081000C2203811C2AFC29175D533D294D2AF7510
:100820009F300208C2C2AFC29575D533D290D2AF05
:10083000759F100208C2203810C2AFC294D29075C2
:10084000D533D2AF759F108079C2AFC290D2947564
:10085000D533D2AF759F308069203811C2AFC293B3
:1008600075D50FD290D2AF759F200208C2C2AFC219
:100870009375D53CD294D2AF759F200208C2203820
:1008800010C2AFC290D29275D50FD2AF759F308093
:1008900031C2AFC294D29275D53CD2AF759F108051
:1008A00021203810C2AFC29575D53CD292D2AF7517
:1008B0009F10800EC2AFC29175D50FD292D2AF7584
:1008C0009F30C22322C295C293C291C294C292C2E7
:1008D0009075D53F22788076FF0876FF0876FF086E
:1008E00076FF0876FF0876FF0876090876FF087617
:1008F00001788C76010876FF0876FF0876FF087687
:10090000FF0876FF0876030876FF0876FF0876FF73
:100910000876250876D008762808765008760408E8
:1009200076FF0876020876FF08767A0876FF087662
:10093000010876010876FF0876FF08760008760041
:1009400022FA75F00CA4ABF0EAC333F8740133F962
:10095000E8C333F8E933F9E8C32BF8E93400F922A6
:100960007888E6C39403D23A5002C23AC238E630DD
:10097000E102D238A23892397886E614900080934A
:1009800078A6F67886E6F53FC394025003753F02D9
:10099000789CE6753EFFB40203753EA0B403037570
:1009A0003E827896E6314188318932789EE631413F
:1009B000883389347897E631418835893611C522E4
:1009C0003035117A007B007CFF7D007E0051278B43
:1009D0005F8A5E22303A227896E6FA7B00789EE6BD
:1009E000FC7D00C3EA33FAEB33FBC3EC33FCED339D
:1009F000FD7E0A51278B618A607896303A02789E94
:100A0000E6FA7B007897E6FC7D007E00303A10C362
:100A1000EA33FAEB33FBC3EC33FCED33FD7E0A51D2
:100A2000278B5F8A5E2222C3EC9EFCED9400FDC3FF
:100A3000EC9AFCED9BFDC3EC9423ED940050047CF8
:100A4000237D00C3EC94FFED940140047CFF7D0105
:100A50007BFF0B7A000AEA7009C3EC33FCED33FD2F
:100A60004152EC8AF0A4AEF0ED8AF0A42E947C40C2
:100A7000E4EAF460DD22D23531C01202E97A007B6B
:100A8000007C101202E1E5522AFA74003BFBDCF311
:100A90007C04C3EB13FBEA13FADCF7FFEB60027F85
:100AA000FFC23531C02278A5E6F954037000E9543D
:100AB0000C7000E954307000E954C0700022E5EF7A
:100AC00020E6037520000520903FFFE52014600616
:100AD000901DFF1460009304600375EF127597DE9C
:100AE0007597AD7581C043FF801202DD75EF027509
:100AF000A90011C57580FF75F1F075A4007580FF20
:100B000075D4FF75900075F23F75A53F759000751F
:100B1000D53F75A60175E34075E20211C5E4F8F60C
:100B2000D8FD11D5D1A278988662753001C2AF1276
:100B300002F11203001202E91203061202E9120383
:100B40000C1202E951A6C2AF78FA79FA308507D9BA
:100B5000FBD8F7021C00316031C07898866211C55D
:100B600075E405758811758E0475890975C8047555
:100B7000910475D84075D90875F781759E037596EF
:100B80000275DA4275DB4275A82175E69075F3109F
:100B9000759B80759D0075D12C75BC5875BB107503
:100BA000E88075B2011202DDD2AF753C00C230128E
:100BB00002F1C2317522001202EDC3E522940A400F
:100BC00024D231C2327522001202EDC3E522940A0A
:100BD0004013D232C2337522001202EDC3E52294D3
:100BE0000A4002D2331202E1203003020B46C2AFA8
:100BF000120300120300120300D2AF1202F1303AC6
:100C000002818F1202E1788CE6C394015002818F39
:100C1000E530C394015002818F7F02D23531C0127A
:100C200002EDC2AFC23531C0AE52C3E552947FD29D
:100C3000AF405C1202DDC2AF120312D2AFDFDC5153
:100C400076C3EF7897F61202F1D1DCF17E7F0AD2FB
:100C50003531C01202EDC2AFC23531C0AE52C3E56C
:100C600052947FD2AF50E61202DDC2AF12030012DF
:100C700002E5120300D2AFDFD65176EF2403789657
:100C8000F61202F1D1DCF1AD1202ED31C061461273
:100C900002ED7801303A027805C3E55298400261CE
:100CA000FEC2AF120312120312120312D2AF1202CB
:100CB000F1753000E4F537F5380537E537F4703E67
:100CC0000538789AE67819146012783214600D7835
:100CD0007D14600878FA146003753800C3E538980D
:100CE000401C11C51202DD153875370078998662EF
:100CF000C2AF120312D2AF789886621202ED1202CE
:100D0000E5E523700261467801C3E5529840AA12D6
:100D100002EDE5237003020B46C2AF11C5E4D2AF6A
:100D2000E4F55CF524F525F53D755C081202DD124D
:100D300003BAE5E820ECFBA8BDA9BEE97001F8887C
:100D40005D1203BE755C08C2AF7559FF120427859A
:100D50005B59855B5AD2AF303A07C238303402D281
:100D600038D228753900117E11A112043F120446B1
:100D700012043F12044612043F1206B51207A112D4
:100D800007EE1204461206A5202C0312035D302C38
:100D9000031203A41207A111111204461206B51280
:100DA00007A111361204461206A51207A111591205
:100DB00004461206B51207A1117E1204461203BAA8
:100DC0001206A51207A111A11203BE120446302873
:100DD00027855B5979187A0CC3E53999400EC228EA
:100DE000D2298A3B855B59855B5A800CC3E55294B6
:100DF000014003020D79C17830291C202B19E53BF5
:100E0000147006C229D22AA179F53BC3E552940198
:100E10004003020D798061753C0078FA79A4E7609F
:100E2000027803C3E55398504FE523604B303A17DF
:100E3000203805203407800F303402800A202B0729
:100E4000D22B855B59A1A778F0302B05855B5978AB
:100E500020C3E548985003020D79302B1BC22BC2EA
:100E600038303402D238D229753B12855B59A179CA
:100E7000053CE5526002C17B753C00C2AF11C575EF
:100E80002400752500D2AF1202ED11C578A4E660EA
:100E900006D294D292D290C3E53C940440026146BB
:100EA00081B4901A0D7820F115E520B4550AA3F10C
:100EB00015E520B4AA02800611D5D1DC801D901A58
:100EC0000378807B0AF115A308DBFA901A0F788C5F
:100ED0007B1AF115A308DBFA901A2922C2AFF1544C
:100EE000F12E901A007410F11AA37401F11AA37470
:100EF00020F11A901A0378807B0AF119A308DBFA13
:100F0000901A0F788C7B1AF119A308DBFAF167F1BC
:100F100045901A2922E493F622E6438F01538FFD70
:100F200075EF0275B7A575B7F1F0538FFE22438FA9
:100F300002438F0175EF0275B7A575B7F1901A0DD1
:100F4000F0538FFC22901A0D7455F11A901A0E74FA
:100F5000AAF11A227A3079D07820901A40F115E55A
:100F600020F709A3DAF7227A3079D0901A40E7F116
:100F70001A09A3DAF9227C051202F1DCFB22C2AFC6
:100F800012030012030612030C1203121202E512DE
:100F9000030012030612030C1203121202E51203DD
:100FA0000012030612030C120312D2AF22C2AF12B8
:100FB000031212030C1203061203001202E51203BD
:100FC0001212030C1203061203001202E51203129E
:0C0FD00012030C120306120300D2AF2221
:1019FD00020ABE100120FFFFFFFFFFFF09FF01FFDD
:101A0D0055AA01FFFFFFFFFF03FFFFFF25D0285061
:0D1A1D0004FF02FF7AFF0101FFFF0000FF40
:101A400023425F4C5F31352320202020202020209E
:101A500023424C48454C492445464D3842313023B9
:101A60002020202020202020202020202020202076
:101C0000C2AFC2D37597DE7597AD7581C075A90057
:101C100043FF80752438752503B1C875EF0243F181
:101C20002053A4DFD28575D4FF75E3407DFA780395
:101C300079E67C10752200752300901DD57B067512
:101C400024987525013085028145208508D8FBD967
:101C5000F9DCF781B7308508D8FBD9F9DCF781B713
:101C6000B188E493A3C39A6004DDC381B7DBDBB121
:101C70007A6002812E7B08E493FAA3B15BDBF87AE9
:101C800030B15B752200752300B17AEAFCEBFDC32D
:101C9000ED94FE400EB17A8A278B28ED30E0048A5D
:101CA000828B83B17A7AC270D8C3ED94FE601350F0
:101CB000CEBD0023EC60097520007521FF020000F5
:101CC0008100A827A9280809D804D90281D4B17EA7
:101CD000EAF281C80D81A3C3ED94035047EDA2E061
:101CE00092007AC5C3E5829400E583941C5092204B
:101CF0000010438F02438F0175B7A575B7F1F0301F
:101D0000001DA827A9280809438F01538FFDD80477
:101D1000D902A11FE275B7A575B7F1F0A3A10E53C3
:101D20008FFC817F7AC1BD030CE493A3FAB13FDC41
:101D3000F8B137817F8181AA22AB23B15BEBFAEA4C
:101D40006222752608C3E52313F523E52213F52245
:101D500050066323A0632201D526EAB1C8B1C87535
:101D6000260AEAF4200102D285300102C285B1C8F8
:101D7000C3134002C201D526EB22B17EEAFB2085C7
:101D800002A17E308502A183752608AE24AF25C34B
:101D9000EF13FFEE13FEB1CCB1C8C3EA13308502D6
:101DA0004480FA30E703632201C3E52313F523E5FA
:101DB0002213F52250066323A0632201D526D9E51C
:101DC0002265236523F52222AE24AF250E0FDEFE09
:101DD000DFFCD20122424C48656C6934373163E83C
:031DE000B1060148
:00000001FF
